:10000000D929A401A5012620C63E031803280A3ECB
:10001000031C0328A2000310240DA000250DA1003D
:10002000200DA10DA4070318A10A2108A507A40DFE
:10003000A50D2208A4070318A50A2620C63E03180A
:1000400024280A3E03180A282408080042283908F0
:10005000A0003708A1000130A200A30164005320D2
:10006000031C4628A20B2E28FF30A30703182E28B6
:10007000A007031CA107031CD4293230A2000030C2
:10008000A3002E286400532003184228A320083020
:10009000A300A4205320A20C4D28A30B4928A42080
:1000A00003142208080038088400360884178004E6
:1000B0008413000535193606FF3E0800A501A4008B
:1000C000B5172730A300103071200330A300E830AB
:1000D0007120A30164307120A3010A30712024082B
:1000E0007C28A2002508A1002408A0009D2120084A
:1000F000031DB513B51B0800303EA6003808840068
:100100000930A70003108920A60CA70B832803142D
:1001100089288413B51D982800083604351D360635
:100120008000841700083604031C36068000A428CB
:1001300000083604031C360635193606800084177D
:1001400036098005A4283517350D0639A000B220E0
:10015000A100A00AB220351F81293513A00002306A
:100160009821812900308A002008820701347534E3
:100170000334153400343C340C34D9346400D420B6
:100180000318BE281921A8010830A3001A21D42081
:100190000318A80AAB1EA801A20CA30BC628AB1A11
:1001A000A2131A2122080800380884003608841790
:1001B0008004841300052B1B3606FF3E0800290827
:1001C0000319D429CF21A903DF28A401A501B51261
:1001D000CF21D33E0319B5162D3EC63E0318E8289D
:1001E0000A3E031CE828A2000310240DA000250DE0
:1001F000A100200DA10DA4070318A10A2108A5073D
:10020000A40DA50D2208A4070318A50AA903031924
:100210001029CF21C63E031810290A3E0318F328DF
:10022000B51E1729A409A509A40A0319A50A2408BB
:10023000D42935172B081F39FF3EA1002A08F53EA7
:100240000318A10A351F81293513A0000230982117
:100250008129A30038088400360950218413A3089B
:100260000319D429F030A50022088038A400F0300A
:10027000A5030319A5000319A3030319D4294029D1
:100280005321030120183608A21F3608A2080319BB
:100290000301A40F4D29800634294E290000372977
:1002A00084178005D429210820040319A00A80306E
:1002B000201AA1062019A106A018A106210DA00D43
:1002C000A10DD42983169B001C141A08D429831667
:1002D0009A001C1555309D00AA309D009C149C1856
:1002E0006F291C11D429A301A200FF30A207031C0F
:1002F000A307031CD4290330A100DF308121752915
:10030000A101E83EA000A109FC30031C8A29A00736
:1003100003188729A0076400A10F872920189029B6
:10032000A01C94290000942908000310A10CA00C23
:10033000FF3E031895292008D429A501A4011030F7
:10034000A600210DA40DA50D2208A4022308031C5C
:10035000230FA5020318B3292208A40723080318B2
:10036000230FA5070310A00DA10DA60BA12920089E
:10037000D4291030A800A101A001A70CA60C031CD1
:10038000C7292208A00723080318230FA107A10CDF
:10039000A00CA50CA40CA80BBD292408D42984000A
:1003A00031088A003008820083130313831264002B
:1003B000080007309F0083161C30850086018312D9
:1003C0003C30BD000530BC000F30BB006400851D13
:1003D000EA295D2C0630B8000430B6000630B500BE
:1003E0000D307D200A307D20C20142086221BA0012
:1003F0000630B8000430B6000630B5003A087D205B
:10040000C20A64004208633C031D072A0E2A6400E6
:100410003A085A3C031D0D2A0E2AF5290630B80069
:100420000430B6000630B5000D307D200A307D2046
:1004300043307D2068307D2067307D2020307D2056
:100440006D307D2073307D2067307D203F307D20F2
:1004500020307D2079307D202F307D206E307D2032
:100460000D307D200A307D200530B8001030B600F8
:100470000630B5001030B9002730B7002720031C24
:100480005D2CC40064004408793C0319482A972A6B
:100490000630B8000430B6000630B5000D307D20BF
:1004A0000A307D2045307D206E307D2074307D20E7
:1004B00020307D206D307D2073307D2067307D20A1
:1004C00020307D2074307D2068307D2065307D2097
:1004D0006E307D2020307D205A307D200D307D20F3
:1004E0000A307D20C2010530B8001030B600063059
:1004F000B5004220C100420883169B0083124108C8
:1005000067210630B8000430B6000630B500410857
:100510007D20640041085A3C031D8F2A0E2AC20A1E
:1005200064004208633C031D962AF529732A0630AD
:10053000B8000430B6000630B5000D307D200A301A
:100540007D200630B8000430B6000630B5000D300E
:100550007D200A307D2020307D2020307D202030FD
:100560007D2045307D2076307D2065307D206E30C9
:100570007D2020307D204F307D2064307D20643010
:100580007D200D307D200A307D206430C200640063
:10059000703042020318052B9C304207B200FF3036
:1005A0000318013EB3000530A600A7013208A200DF
:1005B0003308A300B921C30042086221C5000C30F2
:1005C0004207B200B301B30D32086221C600063003
:1005D000B8000430B6000630B50043085E20203075
:1005E0007D2073307D2065307D2063307D2020307C
:1005F0007D2045085E2020307D2046085E200D309D
:100600007D200A307D20C20FC72A0630B800043092
:10061000B6000630B5000D307D200A307D20063052
:10062000B8000430B6000630B5000D307D200A3029
:100630007D2043307D2068307D2067307D20203054
:100640007D2047307D2050307D2053307D203F304D
:100650007D2020307D2079307D202F307D206E3030
:100660007D200D307D200A307D200530B80010300F
:10067000B6000630B5004220C40064004408793C4E
:100680000319432B5D2C0630B8000430B600063049
:10069000B5000D307D200A307D2035307D202030A2
:1006A0007D2073307D2065307D2063307D202030BB
:1006B0007D2073307D206C307D206F307D20743044
:1006C0007D2073307D202C307D2020307D20303007
:1006D0007D202D307D2035307D2035307D2020302F
:1006E0007D2069307D2066307D2020307D20653082
:1006F0007D2076307D2065307D206E307D2020305D
:100700007D206D307D2069307D206E307D207330FE
:100710007D202C307D2020307D2036307D203030F3
:100720007D202D307D2031307D2031307D203530D1
:100730007D2020307D2069307D2066307D20203076
:100740007D206F307D2064307D2064307D2020301E
:100750007D206D307D2069307D206E307D207330AE
:100760007D200D307D200A307D200630B800043019
:10077000B6000630B5000D307D200A307D20733084
:100780007D2065307D2074307D202F307D206330CA
:100790007D206C307D2072307D203F307D202030E8
:1007A0007D2073307D202F307D2063307D200D3003
:1007B0007D200A307D200530B8001030B6000630AC
:1007C000B5004220C4000630B8000430B600063040
:1007D000B5000D307D200A307D2073307D206530DE
:1007E0007D2063307D203F307D200D307D200A301C
:1007F0007D2064004408733C031DFF2B062C64001D
:100800004408633C031D052C322C972A0530B800A0
:100810001030B6000630B5000120C3007F30C3059C
:100820004308A000A1010530A200A3019D212408D6
:10083000C50064004508003C03191F2C972A430893
:10084000A000A1010530A200A3019D21C2006430D7
:10085000C2070130C500420883169B008312450879
:100860006721972A0530B8001030B6000630B50071
:100870000120C3007F30C3054308A000A10105305B
:10088000A200A3019D212408C50064004508003C86
:1008900003194B2C972A4308A000A1010530A200A0
:1008A000A3019D21C2006430C207C501420883161E
:1008B0009B00831245086721972A0630B800043050
:1008C000B6000630B5000D307D200A307D20723034
:1008D0007D2075307D206E307D202E307D202E30A5
:1008E0007D202E307D203727C727C2014208622194
:1008F000BA0064003A08613C031D7F2CBF256400E8
:100900003A08623C031D852CC62564003A08633C06
:10091000031D8B2CCF2564003A08643C031D912CE9
:10092000D82564003A08653C031D972CE025640037
:100930003A08663C031D9D2CE62564003A08673C96
:10094000031DA32CEF2564003A08683C031DA92C65
:10095000F72564003A08693C031DAF2C00266400AB
:100960003A086A3C031DB52C072664003A086B3C24
:10097000031DBB2C102664003A086C3C031DC12CDF
:10098000182664003A086D3C031DC72C212664001C
:100990003A086E3C031DCD2C282664003A086F3CB3
:1009A000031DD32C2F2664003A08703C031DD92C5C
:1009B000372664003A08713C031DDF2C4026640092
:1009C0003A08723C031DE52C492664003A08733C42
:1009D000031DEB2C512664003A08743C031DF12CD6
:1009E000592664003A08753C031DF72C5F26640005
:1009F0003A08763C031DFD2C672664003A08773CD4
:100A0000031D032D702664003A08783C031D092D50
:100A1000782664003A08793C031D0F2D8126640076
:100A20003A087A3C031D152D8A2664003A08313CA9
:100A3000031D1B2D932664003A08323C031D212D13
:100A40009D2664003A08333C031D272DA726640029
:100A50003A08343C031D2D2DB12664003A08353C7C
:100A6000031D332DBB2664003A08363C031D392D87
:100A7000C52664003A08373C031D3F2DCF2664008D
:100A80003A08383C031D452DD92664003A08393C04
:100A9000031D4B2DE32664003A08303C031D512D05
:100AA000ED2664003A08203C031D572D1B276400E7
:100AB0003A082F3C031D5D2DF72664003A08423C9E
:100AC000031D632D222764003A08433C031D692D52
:100AD000292764003A08443C031D6F2D3027640029
:100AE0003A08483C031D752D372764003A084B3CF3
:100AF000031D7B2DC32764003A084C3C031D812D48
:100B0000412764003A084D3C031D872D3C276400B3
:100B10003A08503C031D8D2DEE2764003A08513CE5
:100B2000031D932DF02764003A08533C031D992DB3
:100B3000CA2764003A08543C031D9F2DDD2764003A
:100B40003A08553C031DA52DC72764003A08573CB9
:100B5000031DAB2D4B2764003A08583C031DB12DF3
:100B6000462764003A085A3C031DB72D5D2CC20A83
:100B700064004208633C031DBE2D5D2C762C0127CA
:100B80000E273D0873213D08732108000E27012719
:100B9000012701273D0873213D08732108000E2716
:100BA00001270E2701273D0873213D087321080006
:100BB0000E27012701273D0873213D0873210800F6
:100BC00001273D0873213D087321080001270127F3
:100BD0000E2701273D0873213D08732108000E27C9
:100BE0000E2701273D0873213D08732108000127C6
:100BF0000127012701273D0873213D0873210800C3
:100C0000012701273D0873213D08732108000127B2
:100C10000E270E270E273D0873213D08732108007B
:100C20000E2701270E273D0873213D087321080078
:100C300001270E27012701273D0873213D08732155
:100C400008000E270E273D0873213D087321080078
:100C50000E2701273D0873213D08732108000E2748
:100C60000E270E273D0873213D0873210800012738
:100C70000E270E2701273D0873213D087321080028
:100C80000E270E2701270E273D0873213D087321EB
:100C9000080001270E2701273D0873213D08732115
:100CA00008000127012701273D0873213D08732112
:100CB00008000E273D0873213D0873210800012715
:100CC00001270E273D0873213D08732108000127E5
:100CD000012701270E273D0873213D0873210800D5
:100CE00001270E270E273D0873213D0873210800B8
:100CF0000E27012701270E273D0873213D08732188
:100D000008000E2701270E270E273D0873213D08F6
:100D1000732108000E270E27012701273D087321A4
:100D20003D087321080001270E270E270E270E27E6
:100D30003D0873213D0873210800012701270E2774
:100D40000E270E273D0873213D0873210800012757
:100D5000012701270E270E273D0873213D08732127
:100D6000080001270127012701270E273D087321CD
:100D70003D087321080001270127012701270127CA
:100D80003D0873213D08732108000E270127012724
:100D9000012701273D0873213D08732108000E2714
:100DA0000E270127012701273D0873213D087321E4
:100DB00008000E270E270E27012701273D08732163
:100DC0003D08732108000E270E270E270E27012746
:100DD0003D0873213D08732108000E270E270E27BA
:100DE0000E270E273D0873213D08732108000E27AA
:100DF000012701270E2701273D0873213D08732194
:100E0000080086140630B8000830B6006E30A20024
:100E10003C08292186103D087321080086140630FD
:100E2000B8000830B6006E30A2003B0829218610B9
:100E30003D08732108003D0873213D0873213D08DA
:100E4000732108007830BD000A30BC001E30BB00A2
:100E500008005430BD000730BC001530BB0008004E
:100E60003C30BD000530BC000F30BB0008008617C9
:100E7000061386120612080086130617861206123B
:100E8000080086130613861606120800861306133A
:100E90008612061608000530B8001030B600BC30C7
:100EA000AA004030AB00BE20523C031D532FBE2091
:100EB0004D3C031D532FBE20433C031D532FBE202A
:100EC0002C3C031D532F0230A900BE30B000B101ED
:100ED000DF200230A900BE30B000B101E520BE0025
:100EE0000230A900BE30B000B101E520BF006400AF
:100EF0003E1C7C2F3C30BF073F08A000A1010530FD
:100F0000A200A3019D212408C50064004508003CFF
:100F100003198B2F9E2F3F08A000A1010530A200CE
:100F2000A3019D21C6006430C60746086221C500A2
:100F300064004508003C03199E2FC22FBF033F08E1
:100F4000A000A1010530A200A3019D212408C50035
:100F500064004508003C0319AE2F4B2F3F08A0004A
:100F6000A1010530A200A3019D21C6006430C6077F
:100F700046086221C50064004508003C0319C12FE2
:100F8000C22F4B2F080086140130C00008008610C5
:100F9000C001080064004008013C031DD82F063042
:100FA000B8000830B6006E30A20053302921DC2F83
:100FB0000330A300E8307421080064004008013CBD
:100FC000031DEB2F0630B8000830B6006E30A200CB
:100FD00008302921ED2F6430732108000614080021
:080FE000061008006300F22F67
:02400E00653F0C
:0A42000076007600760057005A00A1
:1042C80001000000000000000000000000000000E5
:1042D80000000000000000000100000000000000D5
:1042E80000000000000000000000000000000000C6
:00000001FF
